:020000040000FA
:0600000066EF16F012008D
:020006001200E6
:020008000100F5
:06001800B8EF0CF012002D
:02001E000200DE
:1000200008000000FA01000002000000042D00009A
:08003000D701000023000000CD
:08003800D9CFE6FFE1CFD9FFAB
:10004000800EE66EE1EC0AF0E552729E728CFD0EB7
:10005000DBCFE9FFFE0EDBCFEAFFEE52EF04146EBA
:10006000FD0EDBCFE9FFFE0EDBCFEAFF050EE92632
:10007000000EEA22EF04400DF35014100E01436FFE
:10008000FD0EDBCFE9FFFE0EDBCFEAFF020EE92615
:10009000000EEA22EF04166EFD0EDBCFE9FFFE0E26
:1000A000DBCFEAFF030EE926000EEA22EF04080D7B
:1000B000F3CF15F0FD0EDBCFE9FFFE0EDBCFEAFF3D
:1000C000070EE926000EEA22EF50400DF3CF14F0A0
:1000D000FD0EDBCFE9FFFE0EDBCFEAFF060EE926C1
:1000E000000EEA22EF50800DF35014101510161078
:1000F000446FFD0EDBCFE9FFFE0EDBCFEAFF040EFF
:10010000E926000EEA22EF04156EFD0EDBCFE9FFB3
:10011000FE0EDBCFEAFF090EE926000EEA22EF50C1
:10012000400DF3CF14F0FD0EDBCFE9FFFE0EDBCF69
:10013000EAFF080EE926000EEA22EF50800DF35088
:1001400014101510456F7D95E66A0F0EE66EE66E8B
:10015000E66AE66AF80EE66E0E0EE66EF5EC0AF05A
:10016000146E070EE15E1450E66AE66A0F0EE66E44
:10017000E66AE66AFC0EE66E0E0EE66EF5EC0AF036
:10018000146E070EE15E14500E01466B476B4681FC
:10019000E66AE66A010EE66EE66AE66AE00EE66E7A
:1001A0000E0EE66EF5EC0AF0146E070EE15E1450CA
:1001B0000E014683E66AE66A020EE66EE66AE66AC3
:1001C000E40EE66E0E0EE66EF5EC0AF0146E070E07
:1001D000E15E14500E01F40E796F100E716F7269AA
:1001E000200E706EE66AE1EC0AF0E552606A0F01DB
:1001F000306B0E01806BFD0EDBCFE9FFFE0EDBCF17
:10020000EAFFEF50E66EDED8E552010EE552E7CF89
:10021000D9FF1200D9CFE6FFE1CFD9FFE652FD0E9C
:10022000DBCFE9FFFE0EDBCFEAFFEFCFDFFFDF50D2
:10023000120DF3CFE9FFF4CFEAFF000EE926010E1D
:10024000EA22DFCFEFFFFD0EDBCFE9FFFE0EDBCFB3
:10025000EAFFEE52EECF14F0EECF15F0EECF16F02F
:10026000EFCF17F0DF50120DF3CFE9FFF4CFEAFF25
:10027000000EE926010EEA22EE5214C0EEFF15C070
:10028000EEFF16C0EEFF17C0EEFFFD0EDBCFE9FF5D
:10029000FE0EDBCFEAFF050EE926000EEA22EF5044
:1002A000E66EDF50120DF3CFE9FFF4CFEAFF000E48
:1002B000E926010EEA22050EE926000EEA22E552A1
:1002C000E750EF6EFD0EDBCFE9FFFE0EDBCFEAFF5E
:1002D000060EE926000EEA22EECF14F0EECF15F05E
:1002E000EECF16F0EFCF17F0DF50120DF3CFE9FF8E
:1002F000F4CFEAFF000EE926010EEA22060EE926F7
:10030000000EEA2214C0EEFF15C0EEFF16C0EEFF8D
:1003100017C0EEFF010EE552E552E7CFD9FF1200FC
:10032000D9CFE6FFE1CFD9FF020EE126DF6A010E49
:10033000DB6ADB6A320EF36E010EDBCFF4FFF350A3
:10034000F45C33E2E66AFD0EDBCFE9FFFE0EDBCFA5
:10035000EAFF050EE926000EEA22EF50E66EFB0EDC
:10036000DBCFE6FFFC0EDBCFE6FFFD0EDBCFE9FFC8
:10037000FE0EDBCFEAFFEE52EECFE6FFEECFE6FF5A
:10038000EECFE6FFEFCFE6FF5EEC08F0146E080E4E
:10039000E15E1450DF6EDF5008E10B0EE66E74EC88
:1003A00016F0E552010EDB2AC5D7DF50146E020E9F
:1003B000E15C02E2E16AE552E16E1450E552E7CFFA
:1003C000D9FF1200D9CFE6FF0101006BF70E016FD4
:1003D000020E026F036B046B080E056F066B076B52
:1003E000086B096B010E126FF00E136F010E146F84
:1003F000156B166B040E176FF00E186F010E196F48
:100400001A6B1B6B020E246F060E256F020E266FF1
:10041000276B286B080E296F060E2A6F020E2B6FB2
:100420002C6B2D6B030E366F160E376F020E386F66
:10043000396B3A6B080E3B6F160E3C6F020E3D6F28
:100440003E6B3F6B080E486FFA0E496F020E4A6F03
:100450004B6B4C6B080E4D6F4E6B4F6B506B516B73
:10046000010EE552E7CFD9FF1200D9CFE6FFE1CF69
:10047000D9FFE652DF6A0101E151200DF35001017D
:10048000E9110101C66FDAC1C7F10101D9510101BA
:10049000C86FDCC114F0156ADCC1C9F10101DB5180
:1004A0000101CA6FE6C1CBF1CC6BC651C719C8199F
:1004B000C919CA19CB19CC19000ACD6FC60EE66E40
:1004C000010EE66E000EE66E010EE66E29DFE552C5
:1004D000E552E552E552DF6EDF0406E10101E12B52
:1004E000080EE15D01E3E16BDF50E552E552E7CF35
:1004F000D9FF1200D9CFE6FFE1CFD9FF0F0EE126D9
:10050000080EF36EDB6E0E0EDB6AD9500D0FE66E31
:10051000000EDA20E66ED950080FE66E000EDA20E3
:10052000E66ED9CFE6FFDACFE6FFD950090FE66EC7
:10053000000EDA20E66EB1EC09F0146E080EE15EF2
:100540001450E76E0E0EE7CFDBFF0D0EDB50080BED
:100550000101CE6FD950090FE96EDACFEAFFF00E34
:10056000EE181FE1010EEE181CE1EE501AE1EE50FC
:1005700018E1010EF36E0E0EF3CFDBFFE00EDF1479
:10058000E00BE838E8400201C16F1F0EDF140101E3
:10059000E96FC1C2D1F20201D12B080ED15D01E396
:1005A000D16B0E0EDB50146E0F0EE15C02E2E16ABD
:1005B000E552E16E1450E552E7CFD9FF1200D9CFD2
:1005C000E6FFE1CFD9FF110EE126080EF36EDB6ED8
:1005D0000F0EDB6A100EDB6A090EDB6A0A0EDB6A9D
:1005E0000B0EDB6A0C0EDB6A0D0EDB6AD9500E0FA8
:1005F000E66E000EDA20E66ED950080FE66E000EA9
:10060000DA20E66ED9CFE6FFDACFE6FFD950090F40
:10061000E66E000EDA20E66EB1EC09F0146E080EFC
:10062000E15E1450E76E0F0EE7CFDBFF0E0EDB50DE
:10063000080B0101CE6F7792D950090FE96EDACF1E
:10064000EAFFF00EEE180AE1010EEE1807E1EE5097
:1006500005E1EE5003E10101010EE26F146A0F0E95
:10066000156E166A176AD950090FE96EDACFEAFFDC
:10067000EE501416EE501516EE501616EE501716D4
:10068000145039E1010E151836E1165034E11750B7
:1006900032E1090EDBCF00F40A0EDBCF01F40B0EC2
:1006A000DBCF02F40C0EDBCF03F4100EDB6A080E76
:1006B000F36E100EDBCFF4FFF350F45C01E3B4D023
:1006C000D9CF14F0DACF15F0100EDB500F01D9247A
:1006D000E96E000EDA20EA6EEF50E66E100EDB5087
:1006E000EA6A240FE96E040EEA22E552E750EF6E43
:1006F000100EDB2ADCD7146A0F0E156E166A176A05
:10070000D950090FE96EDACFEAFFEE501416EE5019
:100710001516EE501616EE501716145001E089D03B
:10072000020E151801E085D0165001E082D0175056
:1007300001E07FD00F0E146E156A166A176AD95041
:10074000090FE96EDACFEAFFEE501416EE501516D7
:10075000EE501616EE5017160D0E14C0DBFFDB2AF6
:10076000DB50040DF3CFE9FFF4CFEAFF000EE926DA
:10077000040EEA22090EDBCFEEFF0A0EDBCFEEFFFE
:100780000B0EDBCFEEFF0C0EDBCFEEFF100EDB6AA5
:10079000080EF36E100EDBCFF4FFF350F45C26E28C
:1007A000D9CF16F0DACF17F0100EDB500F01D92495
:1007B000E96E000EDA20EA6EEF50E66E0D0EDB50A9
:1007C000080DF3CF14F0F4CF15F0240E1426040E08
:1007D0001522100EDB501424E96E000E1520EA6E6F
:1007E000E552E750EF6E100EDB2AD2D70F0E146ED3
:1007F000156A166A176AD950090FE96EDACFEAFF4F
:10080000EE501416EE501516EE501616EE50171642
:10081000060E141809E1155007E1165005E11750AE
:1008200003E10101010EE46F010EF36E0F0EF3CF31
:10083000DBFF0F0EDB50146E110EE15C02E2E16A89
:10084000E552E16E1450E552E7CFD9FF1200D9CF3F
:10085000E6FFE1CFD9FF030EE126DF6A010EDB6A76
:10086000D950FB0FE96EFF0EDA20EA6ED880FF0E3A
:10087000EE54020EEE54000EEE54000EEE5401E261
:1008800098D0F00E146E156A166A176AD950FB0FCD
:10089000E96EFF0EDA20EA6EEE501416EE501516D1
:1008A000EE501616EE5017160F0E186E196A1A6AC9
:1008B0001B6AD950FB0FE96EFF0EDA20EA6EEE508C
:1008C0001816EE501916EE501A16EE501B16185048
:1008D0001426195015221A5016221B501722020EE8
:1008E00014C0DBFF0F0E146E156A166A176AD95012
:1008F000FB0FE96EFF0EDA20EA6EEE501416EE5092
:100900001516EE501616EE501716060E14183BE18B
:10091000155039E1165037E1175035E1F90EDBCFAC
:10092000E9FFFA0EDBCFEAFFEF50E00BE00BE8380F
:10093000E840E66E020EDB50EA6A000FE96E030E35
:10094000EA22E552E750EF6E010EE76EF90EDBCFBB
:10095000E9FFFA0EDBCFEAFFE750E926000EEA22B4
:10096000EFCFDFFF100EDF14E8380F0BE76E010E3C
:10097000E7CFDBFFEF0EDF14DF6E010EDB5019E077
:100980000101E72B16D0F90EDBCFE9FFFA0EDBCF22
:10099000EAFFEF50E00BE00BE838E840E66E020EAD
:1009A000DB50EA6A000FE96E030EEA22E552E750D7
:1009B000EF6E020EDB50EA6A000FE96E030EEA22C8
:1009C000EFCF14F0020EDB50EA6A600FE96E000E02
:1009D000EA22EF50145C07E1020EDB50EA6A600F76
:1009E000E96E000E21D0020EDB50EA6A000FE96EBC
:1009F000030EEA22EF50E66E020EDB50EA6A600F49
:100A0000E96E000EEA22E552E750EF6E020EDB506F
:100A1000EA6A600FE96E000EEA22EF2A020EDB504E
:100A2000EA6A000FE96E020EEA22EF2A020EDB509C
:100A3000EA6A600FE96E000EEA22EFCF14F0080EAA
:100A4000145C08E3020EDB50EA6A600FE96E000EE8
:100A5000EA22EF6A020E0101E75D03E30101080EDD
:100A6000E96FDF5003E00101080EE96F030EE15C5E
:100A700002E2E16AE552E16EE552E7CFD9FF1200EA
:100A8000D9CFE6FFE1CFD9FFE652F00E146E156A1A
:100A9000166A176AD950FB0FE96EFF0EDA20EA6E6C
:100AA000EE501416EE501516EE501616EE501716A0
:100AB000040ED8901732163215321432E806F9E1D6
:100AC0001450DF6ED950FB0FE96EFF0EDA20EA6E8C
:100AD000F00EEE1827E1010EEE1824E1EE5022E1AF
:100AE000EE5020E1F90EDBCFE9FFFA0EDBCFEAFF93
:100AF000EF50E00BE00BE838E840E66EDF50EA6AC2
:100B0000B20FE96E020EEA22E552E750EF6EF90EDF
:100B1000DBCFE9FFFA0EDBCFEAFFEF501F0B01013D
:100B2000E96F15D0F90EDBCFE9FFFA0EDBCFEAFF54
:100B3000EF50E00BE00BE838E840E66EDF50EA6A81
:100B4000B20FE96E020EEA22E552E750EF6EDF5077
:100B5000EA6AB20FE96E020EEA22EFCF14F0DF501C
:100B6000EA6AC20FE96E020EEA22EF50145C06E157
:100B7000DF50EA6AC20FE96E020E1DD0DF50EA6A4A
:100B8000B20FE96E020EEA22EF50E66EDF50EA6A1B
:100B9000C20FE96E020EEA22E552E750EF6EDF5017
:100BA000EA6AC20FE96E020EEA22EF2ADF50EA6A11
:100BB000D20FE96E020EEA22EF2ADF50EA6AC20F74
:100BC000E96E020EEA22EFCF14F0080E145C07E380
:100BD000DF50EA6AC20FE96E020EEA22EF6AE552BE
:100BE000E552E7CFD9FF1200D9CFE6FFE1CFD9FF19
:100BF000E652DF6ADF50146E156AD890155004E68D
:100C0000A00E145C000E155817E2DF50EA6A000FC0
:100C1000E96E020EEA22EFCF14F0040E145C03E337
:100C20000101080EE96FDF50EA6A000FE96E020E5B
:100C3000EA22EF6ADF2ADED7DF6A100EDF5C17E2F6
:100C4000DF50EA6AD20FE96E020EEA22EFCF14F00B
:100C5000040E145C03E30101080EE96FDF50EA6A39
:100C6000D20FE96E020EEA22EF6ADF2AE6D7E552DA
:100C7000E552E7CFD9FF1200D9CFE6FFE1CFD9FF88
:100C8000060EE126DF6A010EDB6A020EDB6A030E46
:100C9000DB6A040EDB6AF36E050EF3CFDBFFAEC238
:100CA000CFF1AFC2D0F1A5C2D1F1B0C2D2F1A8C28A
:100CB000D3F1B1C2D4F1ABC2D5F1ACC2D6F10201CD
:100CC000AF51E66ED950010FE96EDACFEAFFE55277
:100CD000E750EE6EED6A010EDBCF14F0020E14C089
:100CE00015F0146A010E14C0DBFF020E15C0DBFF05
:100CF000AE51E76E010EDBCF14F0020EDBCF15F024
:100D0000E7501412010E14C0DBFF020E15C0DBFF0A
:100D1000010EDB2A020E01E3DB2A030EDB6A040E5E
:100D2000DB6A030EDBCF14F0040EDBCF15F0010EEF
:100D3000DBCF16F0020EDBCF17F01450165C155007
:100D400017580CE3050EDBCFE6FF46EC16F0E55234
:100D5000030EDB2A040EE5E3DB2AE3D7CF0EE66EB3
:100D6000010EE66E480EE66E010EE66E90EC01F0A6
:100D7000E552E552E552E552DF6E010EF36E030EC9
:100D8000F3CFDBFF040EDB6A020EF36E030EF3CF2C
:100D9000DBFF040EDB6ADF50146E060EE15C02E23C
:100DA000E16AE552E16E1450E552E7CFD9FF120037
:100DB000D9CFE6FFE1CFD9FF1B0EE126080EDB6A93
:100DC0000E0EF36E090EF3CFDBFF0A0EDB6A0B0E7D
:100DD000DB6A080EF36E0C0EF3CFDBFF0D0EDB6A41
:100DE0000E0EDB6A0F0EDB6A100EDB6AD950110F94
:100DF000E66E000EDA20E66ED9500C0FE66E000E9D
:100E0000DA20E66ED9CFE6FFDACFE6FFD9500D0F34
:100E1000E66E000EDA20E66EB1EC09F0146E080EF4
:100E2000E15E1450E76E0B0EE7CFDBFF110EDB50D7
:100E3000080B0101CE6FD9500D0FE96EDACFEAFF32
:100E4000EE5052E1030EEE184FE1EE504DE1EE5040
:100E50004BE1070EDBCFE6FF060EDBCFE6FF050E0C
:100E6000DBCFE6FF040EDBCFE6FF030EDBCFE6FFB2
:100E7000020EDBCFE6FF010EDB50DF18E552E7186C
:100E8000E552E718E552E718E552E718E552E7188A
:100E9000E552E718E76E0A0EE7CFDBFF080EDB50DE
:100EA000F36E0A0EDB50F35C15E10101800EE56F75
:100EB000E66AF60EE66E0D0EE66EE66AE66AF80E75
:100EC000E66E0E0EE66EF5EC0AF0146E070EE15EAD
:100ED00014500AD0090EDB50F36E0A0EDB50F35C9F
:100EE00003E101010A0EE56F0101E5510A0A01E182
:100EF0008ED08A0A01E092D0D9500D0FE96EDACF78
:100F0000EAFF090EEE1806E1030EEE1803E1EE50BB
:100F100001E1EE5002E0000E01D0010E146ED95036
:100F20000D0FE96EDACFEAFF080EEE1806E1030EA8
:100F3000EE1803E1EE5001E1EE5002E0000E01D0A8
:100F4000010E14106BE0120EDB6A0C0EDB50F36E18
:100F5000120EDBCFF4FFF350F45C20E2D9CF16F091
:100F6000DACF17F0120EDB500F01D924E96E000E14
:100F7000DA20EA6EEF50E66ED950130F146EDACF16
:100F800015F0120EDB501424E96E000EDA20EA6E22
:100F9000E552E750EF6E120EDB2AD7D7D9500D0F6E
:100FA000E96EDACFEAFF080EEE1814E1030EEE1830
:100FB00011E1EE500FE1EE500DE1D950130FE66E46
:100FC000000EDA20E66EE66AA2EC12F0E552E55277
:100FD000E55224D0D9500D0FE96EDACFEAFF090EA1
:100FE000EE181CE1030EEE1819E1EE5017E1EE5079
:100FF00015E1D950130FE66E000EDA20E66E080EEA
:10100000E66EA2EC12F0E552E552E55201D034DE74
:101010000101200EE96F0101010EE56F0B0EDB509F
:10102000146E1B0EE15C02E2E16AE552E16E1450BF
:08103000E552E7CFD9FF1200E1
:08103800800EE66EC2DAE552FB
:101040000E01010E436FF80E446F440E456F200EE3
:10105000706E729E728C606A0F01306B0E01806B35
:10106000906BA06BB06BC06BD06BF80E7D6F880E71
:10107000E06F220EE16FE46F080EE56F140EE86F6B
:10108000050EE96F070E466F476B716B110E726F9D
:10109000736F746B756B766B776B786B500E796FC3
:1010A000050E7A6F7B6B7B6BF869F969F997FC6BBE
:1010B000FD6BFD97E66A85DAE5521200D9CFE6FFAF
:1010C000E1CFD9FF1A0EE126D950060FE96EDACF2B
:1010D000EAFF200EEE6E0F0EED6ED950080FE96E8E
:1010E000DACFEAFF100EEE6E0F0EED6ED9500A0F3A
:1010F000E96EDACFEAFF000EEE6E0F0EED6ED950FC
:101100000C0FE96EDACFEAFF800EEE6E0E0EED6E7A
:10111000D9500E0FE96EDACFEAFF900EEE6E0E0E8A
:10112000ED6ED950100FE96EDACFEAFFA00EEE6E29
:101130000E0EED6ED950120FE96EDACFEAFFB00E47
:10114000EE6E0E0EED6ED950140FE96EDACFEAFF97
:10115000C00EEE6E0E0EED6ED950160FE96EDACFA0
:10116000EAFFD00EEE6E0E0EED6E0E017D417F0B8E
:10117000E76E190EE7CFDBFFDF6ADF50146E156AEA
:10118000080E145C000E155801E3DED0D950060F8E
:10119000146EDF50020D1450F324E96EDA50F4207F
:1011A000EA6E020EEECFDBFF030EEDCFDBFF020E89
:1011B000DBCF08F0030EDBCF09F0040E08C0DBFF25
:1011C000050E09C0DBFFDF50020810E2190EDBCF6D
:1011D000F3FFF390F342F3CFDBFFD950190FE96E21
:1011E000DACFEAFFEF50010B01E1ACD0020EDBCF0A
:1011F000E9FF030EDBCFEAFFEF50080B01E0A2D0BE
:10120000FC0E146E020EDBCFE9FF030EDBCFEAFF0C
:101210001450EF16F70EDB50030B146E020EDBCFEB
:10122000E9FF030EDBCFEAFF1450EF12F70EDBAC41
:1012300004D0F80EDB50400902D0F80EDB50E76E08
:10124000180EE7CFDBFF050EE76E020EDBCFE9FFDE
:10125000030EDBCFEAFFE750E926000EEA22180E64
:10126000DBCFEFFFF70EDBAA06D0010EF36E180EF0
:10127000F3CFDBFF02D0180EDB6ADBCFE6FFD950DD
:10128000FB0FE96EFF0EDA20EA6EEECFE6FFEECF3F
:10129000E6FFEECFE6FFEFCFE6FF010EE76E020EB0
:1012A000DBCF14F0030EDBCF15F0E7501426000E51
:1012B000152214C0E6FF15C0E6FF97D9166E070E7B
:1012C000E15E1650D950020FE96EDACFEAFF060E42
:1012D000EE26000EED22010EDB6AF80EDB50F36EF7
:1012E000010EDBCFF4FFF350F45C1AE2F90EDBCF12
:1012F000E9FFDB2AFA0EDBCFEAFF01E3DB2AEF503E
:10130000E66E020EDBCFE9FFDB2A030EDBCFEAFF3E
:1013100001E3DB2AE552E750EF6E010EDB2ADDD751
:10132000040EDBCFE9FF050EDBCFEAFFEF50040B25
:1013300007E1040EDBCFE9FF050EDBCFEAFFEF8606
:10134000010E03D0DF2A19D7000E146E1A0EE15CCD
:1013500002E2E16AE552E16E1450E552E7CFD9FFAF
:101360001200D9CFE6FFE1CFD9FF060EE126010139
:10137000FC6B60AE04D0600EDE6E0F0E43D00F012A
:1013800030AF04D0300EDE6E0F0E3CD00E017D511A
:10139000040B07E18051800B04E0800EDE6E0E0E20
:1013A00031D07D51080B07E19051800B04E0900E85
:1013B000DE6E0E0E27D07D51100B07E1A051800B81
:1013C00004E0A00EDE6E0E0E1DD07D51200B07E155
:1013D000B051800B04E0B00EDE6E0E0E13D07D51C6
:1013E000400B07E1C051800B04E0C00EDE6E0E0E14
:1013F00009D07D51800B13E1D051800B10E0D00E4D
:10140000DE6E0E0EDD6EDECFE9FFDDCFEAFFEF50C0
:101410001F0B0101FC6F779271AC0BD002D0000E54
:10142000C4D0F70EDBCFE9FFF80EDBCFEAFFEF8683
:10143000719CD9CFE9FFDACFEAFF020EEECFDBFFD6
:10144000030EEDCFDBFFF70EDBCFE9FFF80EDBCFAE
:10145000EAFFEF6ADECFE9FFDDCFEAFF050EE926FE
:10146000000EEA22050EEFCFDBFFDB500F0BE66E1E
:10147000F90EDBCFE9FFFA0EDBCFEAFFE552E750CA
:10148000EF6ED950050FE96EDACFEAFFEF50400B4F
:1014900007E0F70EDBCFE9FFF80EDBCFEAFFEF8CBA
:1014A000DECFE9FFDDCFEAFF020EE926000EEA22D9
:1014B000050EEFCFDBFFD950050FE96EDACFEAFF5B
:1014C000EF50080B0DE0F70EDBCFE9FFF80EDBCF96
:1014D000EAFFEF8A010EF36E050EF3CFDBFF02D0B9
:1014E000050EDB6ADBCFE6FFFD0EDBCFE6FFFE0E6F
:1014F000DBCFE6FFDECF14F0DDCF15F0010E1426B2
:10150000000E152214C0E6FF15C0E6FF46D9166E80
:10151000050EE15E1650060EDE26000EDD22F90EE7
:10152000DBCFE9FFFA0EDBCFEAFF050EEFCFDBFFE3
:10153000040EDB6ADBCF14F0156A14BE1568050EC5
:10154000DB50000115AE02D0D89003D0145C000E21
:10155000155819E2DFCFE9FFDF2A010EDBCFEAFFE2
:1015600001E3DB2AEF50E66EFB0EDBCFE9FFDB2A5F
:10157000FC0EDBCFEAFF01E3DB2AE552E750EF6E1A
:10158000040EDB2AD7D777AE08D0F70EDBCFE9FF02
:10159000F80EDBCFEAFFEF88779E020EDBCFE9FF84
:1015A000030EDBCFEAFFEF9E010E146E060EE15C28
:1015B00002E2E16AE552E16E1450E552E7CFD9FF4D
:1015C0001200D9CFE6FFE1CFD9FF1F0E6F16FE0E36
:1015D000DB506F12E00E6F14146EFE0EDB50145CC5
:1015E000F9E1E552E7CFD9FF1200D9CFE6FFE1CF0D
:1015F000D9FF020EE126D950F90F146EFF0EDA2042
:1016000014C0DEFFDD6EF80EDB50146E156AE85074
:10161000151031E1DECFE9FFDDCFEAFFEF50E84002
:10162000E840E8401F0BE66EFD0EDBCFE9FFFE0E43
:10163000DBCFEAFFE552E750EF6EDECFE9FFDDCF0B
:10164000EAFFEE52EF50200DF3CF14F0FD0EDBCF8A
:10165000E9FFFE0EDBCFEAFFF350EF12FD0EDB2AAF
:10166000FE0E01E3DB2ADECFE9FFDDCFEAFFEF501C
:10167000200DF3507ED0DECFE9FFDDCFEAFF020E72
:10168000E926000EEA22EF50E00BE838E840E66E6B
:10169000FD0EDBCFE9FFFE0EDBCFEAFFE552E750A0
:1016A000EF6EDECFE9FFDDCFEAFF030EE926000E85
:1016B000EA22EF50080DF3CF14F0FD0EDBCFE9FF67
:1016C000FE0EDBCFEAFFF350EF12FD0EDB2AFE0E1B
:1016D00001E3DB2ADECFE9FFDDCFEAFF020EE926D8
:1016E000000EEA22EF50080DF350E00BE66EFD0EFF
:1016F000DBCFE9FFFE0EDBCFEAFFE552E750EF6EEE
:10170000FD0EDBCFE9FFFE0EDBCFEAFFEF86DECF7B
:10171000E9FFDDCFEAFF020EE926000EEA22EF50D4
:10172000030B146EFD0EDBCFE9FFFE0EDBCFEAFFED
:101730001450EF12FD0EDB2AFE0E01E3DB2ADECF92
:10174000E9FFDDCFEAFFEE52EF50E66EFD0EDBCF94
:10175000E9FFFE0EDBCFEAFFE552E750EF6EFD0E2C
:10176000DB2AFE0E01E3DB2ADECFE9FFDDCFEAFF55
:10177000EF50E66EFD0EDBCFE9FFFE0EDBCFEAFF9A
:10178000E552E750EF6E020EE15C02E2E16AE552DB
:10179000E16EE552E7CFD9FF1200D9CFE6FFE1CFE6
:1017A000D9FF020EE126FB0EDBCFDEFFDBCFDDFF34
:1017B000FA0EDB50156AE85015104CE1FD0EDBCF38
:1017C000E9FFFE0EDBCFEAFFEF50080DF350E66EA7
:1017D000DECFE9FFDDCFEAFFE552E750EF6EFD0E09
:1017E000DBCFE9FFFE0EDBCFEAFFEF50E00BE8387E
:1017F000E840E66EDECFE9FFDDCFEAFFEE52E552CC
:10180000E750EF6EFD0EDB2AFE0E01E3DB2AFD0E34
:10181000DBCFE9FFFE0EDBCFEAFFEF50E00BE8384D
:10182000E840DECFE9FFDDCFEAFFE850EF12DECF80
:10183000E9FFDDCFEAFF020EE926000EEA22EF6A99
:10184000DECFE9FFDDCFEAFF030EE926000EEA2234
:10185000EF6A84D0FD0EDBCFE9FFFE0EDBCFEAFF9F
:10186000EF50200DF350E66EDECFE9FFDDCFEAFF4B
:10187000020EE926000EEA22E552E750EF6EFD0E59
:10188000DBCFE9FFFE0EDBCFEAFFEF50E840E84098
:10189000E8401F0BE66EDECFE9FFDDCFEAFF030E67
:1018A000E926000EEA22E552E750EF6EFD0EDB2A34
:1018B000FE0E01E3DB2AFD0EDBCFE9FFFE0EDBCFE0
:1018C000EAFFEF50030B146EDECFE9FFDDCFEAFF36
:1018D000020EE926000EEA221450EF12FD0EDBCFB5
:1018E000E9FFFE0EDBCFEAFFEF50E00BE840E840F7
:1018F000E8401F0B146EDECFE9FFDDCFEAFF020EDA
:10190000E926000EEA221450EF12FD0EDB2AFE0E2D
:1019100001E3DB2AFD0EDBCFE9FFFE0EDBCFEAFFA2
:10192000EF50E66EDECFE9FFDDCFEAFFEE52E55283
:10193000E750EF6EFD0EDB2AFE0E01E3DB2AFD0E03
:10194000DBCFE9FFFE0EDBCFEAFFEF50E66EDECF26
:10195000E9FFDDCFEAFFE552E750EF6E020EE15CF2
:1019600002E2E16AE552E16EE552E7CFD9FF1200EB
:10197000DACFE4FFE2CFDAFFE9CFE4FFEACFE4FF1A
:10198000F6CFE4FFF7CFE4FFF5CFE4FFF3CFE4FFBA
:10199000F4CFE4FFFACFE4FF00EE00F0140EE80409
:1019A00003E3EECFE4FFFBD700EE14F00E0EE804E5
:1019B00003E3EECFE4FFFBD7E6529D50010B51E06D
:1019C0009E50010B4EE0B20ECF6ECE6A9E90F6C1D5
:1019D00022F0F7C123F0F8C124F0F9C125F00A0E76
:1019E0000B6E0C6A0D6A0E6AF6C106F0F7C107F0BD
:1019F000F8C108F0F9C109F049EC15F002500310E4
:101A00000410051002E10101D781F6C122F0F7C1EF
:101A100023F0F8C124F0F9C125F0640E0B6E0C6AB6
:101A20000D6A0E6AF6C106F0F7C107F0F8C108F0BA
:101A3000F9C109F049EC15F002C022F003C023F00F
:101A400004C024F005C025F0025003100410051056
:101A500002E10101D7830101F62B000EF723F823E1
:101A6000F9237750020B10E07650020B0DE00101D4
:101A7000F46BF56BDFEC02F00101E20505E135ECFA
:101A800002F00101E26BE36BE55200EE21F00E0E75
:101A9000E80403E3E5CFEDFFFBD700EE13F0140EEF
:101AA000E80403E3E5CFEDFFFBD7E5CFFAFFE5CF91
:101AB000F4FFE5CFF3FFE5CFF5FFE5CFF7FFE5CF87
:101AC000F6FFE5CFEAFFE5CFE9FFE5CFDAFF11004A
:101AD000D9CFE6FFE1CFD9FFE652D050DF6E000E3E
:101AE000DB94DB9CDB9EDF501B0A0EE0300A0BE030
:101AF000110A08E0020A05E00B0A01E006D0040022
:101B000005D004D003D002D001D000D03F0ED012B7
:101B1000D398D38AD38C9B9CC26A100EC16E920E4E
:101B2000C06E0F01030E5D6F0F015C6BC28092806F
:101B30009282898A929AFB0E936E8B8094908B92FC
:101B400094928B9494949496949A8B9C949CF00E7B
:101B5000C6140209C66EC698C68AC79C9E96CD88D2
:101B6000CD8A9F909D809E90CD82CD80ADC2EAF1BE
:101B7000EA0EE66E010EE66E1CEC00F0E552E55250
:101B8000F28EF28CFE0EDBCFE9F1E552E552E7CFA3
:101B9000D9FF1200D9CFE6FFE1CFD9FF120EE1261F
:101BA0000E0EDB6A0F0EDB6A100EDB6A110EDB6AAB
:101BB0000101E951100A01E131D2180A01E128D2EC
:101BC0000C0A01E1F1D0060A01E1E0D0220A01E1AC
:101BD0008DD0210A01E050D27AEC02F0040E01010E
:101BE000E95D01E082D00101D880DE5104E7EC0E0E
:101BF000DD5DFF0EDE5902E3000E01D0010E146E12
:101C00000101DE3504E2DD511408000EDE5502E369
:101C1000000E01D0010E141000E0DF6A020EDF5C3E
:101C200059E2DFCFE6FF17EC15F0E552F3CF14F0E1
:101C3000F4CF15F0166A176A15AE02D01668176849
:101C40000E0E14C0DBFF0F0E15C0DBFF100E16C00A
:101C5000DBFF110E17C0DBFFD9500E0FE96EDACF94
:101C6000EAFFD890030EEB50000A08E6440EEE5C43
:101C7000090EEE58000EEE58000EEE5802E3000E6C
:101C800001D0010E146E0E0EDBCF07F00F0EDBCF6E
:101C900008F0100EDBCF09F0110EDBCF0AF00A348A
:101CA000000E0A1809E6D8803E0E07540A0E0854A2
:101CB000000E0954000E0A5402E3000E01D0010E7A
:101CC000141006E00101020EE66F0101080EE96F33
:101CD000DF2AA4D70101E65102E18B828B8478923E
:101CE000768277920E010F0E7E6FC7D1E66A71EC95
:101CF00012F0E5520201E26F0101020EE96FAA0E35
:101D00000201E25D00E0E9C1E6FFE2DEE552DF6AE2
:101D1000100EDF5C17E2DF50EA6AB20FE96E020EC6
:101D2000EA22EF6ADF50EA6AC20FE96E020EEA2287
:101D3000EF6ADF50EA6AD20FE96E020EEA22EF6A1A
:101D4000DF2AE6D7DF6ADF50146E156AD890155087
:101D500004E6A00E145C000E155817E2DF50EA6A84
:101D6000000FE96E030EEA22EF6ADF50EA6A600FA5
:101D7000E96E000EEA22EF6ADF50EA6A000FE96EB0
:101D8000020EEA22EF6ADF2ADED777D148EC10F0A4
:101D9000DBC1DDF1DCC1DEF1D9C1DFF1DAC1E0F197
:101DA0000101010EE96F69D10101D751010B08E072
:101DB0000101D7910101F42B000EF52348EC10F03E
:101DC0000101E851156A2C0F146E010E1522010154
:101DD000F451145CF551155804E20101E82B8B7C99
:101DE0000AD001010A0ED880F455000EF55503E221
:101DF0000101080EE96F0101D751020B66E00101F4
:101E0000D7930101E76BF4EC05F0DF6A020EDF5CAB
:101E100059E2DFCFE6FF17EC15F0E552F3CF14F0EF
:101E2000F4CF15F0166A176A15AE02D01668176857
:101E30000E0E14C0DBFF0F0E15C0DBFF100E16C018
:101E4000DBFF110E17C0DBFFD9500E0FE96EDACFA2
:101E5000EAFFD890030EEB50000A08E6440EEE5C51
:101E6000090EEE58000EEE58000EEE5802E3000E7A
:101E700001D0010E146E0E0EDBCF07F00F0EDBCF7C
:101E800008F0100EDBCF09F0110EDBCF0AF00A3498
:101E9000000E0A1809E6D8803E0E07540A0E0854B0
:101EA000000E0954000E0A5402E3000E01D0010E88
:101EB000141006E00101020EE66F0101080EE96F41
:101EC000DF2AA4D70101010EE36F0101E40501E05F
:101ED0009ED00101E46B010EDB6A090EF36E010E68
:101EE000DBCFF4FFF350F45C01E391D0010EDB5043
:101EF000040DF3CFE9FFF4CFEAFF000EE926040E4C
:101F0000EA22020EEECFDBFF030EEECFDBFF040E64
:101F1000EECFDBFF050EEECFDBFFDF6A080EDF5CE6
:101F200025E2010EDB50080DF3CF16F0F4CF17F0C9
:101F3000240E1626040E1722DF500F011624E96E18
:101F4000000E1720EA6EEF50E66ED950060F146EA1
:101F5000DACF15F0DF500F011424E96E000E1520C2
:101F6000EA6EE552E750EF6EDF2AD8D7146A0F0EFB
:101F7000156E166A176AD950020FE96EDACFEAFFBA
:101F8000EE501416EE501516EE501616EE501716AB
:101F9000145006E1010E151803E1165001E1175027
:101FA0001AE1D950060FE66E000EDA20E66ED9501F
:101FB000020FE96EDACFEAFFEECFE6FFEECFE6FFE3
:101FC000EECFE6FFEFCFE6FF40EC05F0146E060E15
:101FD000E15E145019D0D950060FE66E000EDA20DB
:101FE000E66ED950020FE96EDACFEAFFEECFE6FFD8
:101FF000EECFE6FFEECFE6FFEFCFE6FF27EC04F0F3
:10200000146E060EE15E1450010EDB2A66D735D041
:102010008B948B920101040EE96F2FD00101E5052D
:1020200028E1F29EF29C76920101040EE56FE66AC9
:10203000E6680D0EE66EE66AE66AF80EE66E0E0ECD
:10204000E66EF5EC0AF0146E070EE15E14500E0118
:102050004681E66AE66A010EE66EE66AE66AE00E28
:10206000E66E0E0EE66EF5EC0AF0146E070EE15EFB
:102070001450D8EC06F001D000D00400120EE15C40
:1020800002E2E16AE552E16EE552E7CFD9FF1200C4
:10209000D9CFE6FFE1CFD9FF0A0EE126DE6ADD6A7D
:1020A000020EDB6A030EDB6A040EDB6A050EDB6AD6
:1020B000060EDB6A070EDB6A080EDB6A090EDB6AB6
:1020C000DE6ADD6ADECF14F0DDCF15F0400E145C61
:1020D000000E15582DE2FFEC13F0F3CF14F0F4CFFF
:1020E00015F0166A176AD950020FE96EDACFEAFFC7
:1020F000F350EE261550EE221650EE221750EE2227
:102100007CEC14F0F4CF15F0166A176AD950060F5C
:10211000E96EDACFEAFFF350EE261550EE221650A4
:10212000EE221750EE22DF2A010ECCE3DB2ACAD7BB
:10213000060EDBCF14F0070EDBCF15F0080EDBCF59
:1021400016F0090EDBCF17F0060ED89017321632B4
:1021500015321432E806F9E1060E14C0DBFF070E53
:1021600015C0DBFF080E16C0DBFF090E17C0DBFF32
:10217000060EDBCF06F0070EDBCF07F0080EDBCF35
:1021800008F0090EDBCF09F00A0E0B6E0C6A0D6A1F
:102190000E6AEAEC15F0060E02C0DBFF070E03C064
:1021A000DBFF080E04C0DBFF090E05C0DBFF060ED7
:1021B000DBCF14F0070EDBCF15F0080EDBCF16F0E7
:1021C000090EDBCF17F0070ED890173216321532F2
:1021D0001432E806F9E1060E14C0DBFF070E15C045
:1021E000DBFF080E16C0DBFF090E17C0DBFF060E73
:1021F000DBCF06F0070EDBCF07F0080EDBCF08F0D1
:10220000090EDBCF09F0BB0E0B6E0C6E0D6A0E6A69
:10221000EAEC15F0060E02C0DBFF070E03C0DBFF81
:10222000080E04C0DBFF090E05C0DBFF060EDBCF86
:1022300014F0070EDBCF15F0080EDBCF16F0090EF9
:10224000DBCF17F00B0ED89017321632153214323E
:10225000E806F9E1060E14C0DBFF070E15C0DBFF30
:10226000080E16C0DBFF090E17C0DBFF060EDBCF22
:1022700014F0070EDBCF15F0080EDBCF16F0090EB9
:10228000DBCF17F0AB0E145EEA0E155A000E165A8D
:10229000175A060E14C0DBFF070E15C0DBFF080E31
:1022A00016C0DBFF090E17C0DBFF060EDBCF06F002
:1022B000070EDBCF07F0080EDBCF08F0090EDBCFEF
:1022C00009F00A0E0B6E0C6A0D6A0E6A49EC15F0E5
:1022D000060E06C0DBFF070E07C0DBFF080E08C0B6
:1022E000DBFF090E09C0DBFFDDC118F0DEC119F00C
:1022F0001A6A1B6A19AE02D01A681B68D950060FF9
:10230000E96EDACFEAFF1850EE5C146E1950EE5801
:10231000156E1A50EE58166E1B50EE58176E060EBC
:1023200014C0DBFF070E15C0DBFF080E16C0DBFF75
:10233000090E17C0DBFF060EDBCFDBF1070EDBCF8C
:10234000DCF1020EDBCF14F0030EDBCF15F0040E30
:10235000DBCF16F0050EDBCF17F0060ED890173244
:10236000163215321432E806F9E1020E14C0DBFF12
:10237000030E15C0DBFF040E16C0DBFF050E17C0F1
:10238000DBFF020EDBCF06F0030EDBCF07F0040EFF
:10239000DBCF08F0050EDBCF09F00A0E0B6E0C6ADE
:1023A0000D6A0E6AEAEC15F0020E02C0DBFF030EA6
:1023B00003C0DBFF040E04C0DBFF050E05C0DBFF1E
:1023C000020EDBCF14F0030EDBCF15F0040EDBCFD3
:1023D00016F0050EDBCF17F0020ED890173216322A
:1023E00015321432E806F9E1020E14C0DBFF030EC9
:1023F00015C0DBFF040E16C0DBFF050E17C0DBFFA8
:10240000020EDBCF06F0030EDBCF07F0040EDBCFAE
:1024100008F0050EDBCF09F0FB0E0B6E090E0C6EFB
:102420000D6A0E6AEAEC15F0020E02C0DBFF030E25
:1024300003C0DBFF040E04C0DBFF050E05C0DBFF9D
:10244000020EDBCF14F0030EDBCF15F0040EDBCF52
:1024500016F0050EDBCF17F0080ED89017321632A3
:1024600015321432E806F9E1020E14C0DBFF030E48
:1024700015C0DBFF040E16C0DBFF050E17C0DBFF27
:10248000020EDBCF06F0030EDBCF07F0040EDBCF2E
:1024900008F0050EDBCF09F00A0E0B6E0C6A0D6A10
:1024A0000E6A22EC16F0020E06C0DBFF030E07C018
:1024B000DBFF040E08C0DBFF050E09C0DBFF020EC8
:1024C000DBCFD9F1030EDBCFDAF1F36AF46A0A0E3F
:1024D000E15C02E2E16AE552E16EE552E7CFD9FF45
:0224E0001200E8
:0E24E200D9CFE6FFE1CFD9FF020EE126010EB1
:1024F000DB6ADE52120EDD6EFE0EDB50DF6EDF6A2F
:10250000010EDB50DF5C0EE2DF50746E7F9E7F8039
:10251000DF50EA6AA00FE96E020EEA2273CFEFFFE6
:10252000DF2AEED70201F00EAD6FA051146E020E3D
:10253000E15C02E2E16AE552E16E1450E552E7CF58
:10254000D9FF1200D9CFE6FFE1CFD9FF090EE1266E
:10255000010EDB6A020EDB6A030EDB6A040EDB6A25
:10256000050EDB6A060EDB6A070EDB6A080EDB6A05
:10257000FE0EDB5027E1010EDB6A080EF36E010E42
:10258000DBCFF4FFF350F45C01E32FD1010EDB50FD
:10259000E76EFC0EDBCFE9FFFD0EDBCFEAFFE75075
:1025A000E926000EEA22EF50E66E010EDB28EA6A09
:1025B000A00FE96E020EEA22E552E750EF6E010E1F
:1025C000DB2ADBD7FE0EDB50080801E00ED1010E3E
:1025D000DB6A040EF36E010EDBCFF4FFF350F45C04
:1025E0001DE2010EDB50E76EFC0EDBCFE9FFFD0EB6
:1025F000DBCFEAFFE750E926000EEA22EF50E66E55
:10260000010EDB50090FEA6AA00FE96E020EEA2202
:10261000E552E750EF6E010EDB2ADBD70201AA0E6E
:10262000A06FF00EAD6F300EA15D1A6E1B6A300EFA
:10263000A25D1C6E1D6A0A0E086E096A1CC00DF0B0
:102640001DC00EF07DEC15F01A500624186E1B50BC
:102650000720196E300E0201A35D1E6E1F6A640E04
:10266000086E096A1EC00DF01FC00EF07DEC15F05B
:1026700018500624166E19500720176E300E0201EE
:10268000A45D206E216AE80E086E030E096E20C05C
:102690000DF021C00EF07DEC15F016500624146EDE
:1026A00017500720156EFF0E1416000E1516030E98
:1026B00014C0DBFF040E15C0DBFF300E0201A15D6C
:1026C0001A6E1B6A300EA25D1C6E1D6A0A0E086E21
:1026D000096A1CC00DF01DC00EF07DEC15F01A50FB
:1026E0000624186E1B500720196E300E0201A35DE0
:1026F0001E6E1F6A640E086E096A1EC00DF01FC0B0
:102700000EF07DEC15F018500624166E19500720B7
:10271000176E300E0201A45D206E216AE80E086E6D
:10272000030E096E20C00DF021C00EF07DEC15F0F7
:102730001650062417500720146E156A050E14C093
:10274000DBFF060E15C0DBFF300E0201A75D0A0D90
:10275000300EA65DF324E76E070EE7CFDBFF300EE9
:10276000AA5D0A0D300EA95DF324E76E080EE7CFCF
:10277000DBFF030EDBCFAEF2050EDBCFAFF2070EB1
:10278000DBCFB0F2080EDBCFB1F2120EF36E020E09
:10279000F3CFDBFF010EDB6A020EDB50F36E010E9E
:1027A000DBCFF4FFF350F45C20E2010EDB50746EDB
:1027B000010EDB50EA6AA00FE96E020EEA22EF502A
:1027C000736E7F9E7F9C7F84F250DF6EF26A550E9F
:1027D0007E6EAA0E7E6E7F82DF50F26E7F94B7AC63
:1027E000FED7B79C010EDB2AD7D7090EE15C02E2C7
:0E27F000E16AE552E16EE552E7CFD9FF120033
:0227FE00D9CF31
:10280000E6FFE1CFD9FF060EE126020EDB6A030EDA
:10281000DB6A040EDB6A050EDB6A899A040EDB6A4A
:10282000280EF36E040EDBCFF4FFF350F45C05E2E8
:10283000050EDB2A040EDB2AF3D7050EDB6AC96A14
:102840009EA6FED79E96C950DF6EC96A9EA6FED789
:102850009E96010EC9CFDBFF3F0EDF14E66ED95006
:10286000020FE96EDACFEAFFE552E750EE6EED6A4D
:10287000020EDBCF14F0030E14C015F0146A020E22
:1028800014C0DBFF030E15C0DBFF010EDB50E76E4B
:10289000020EDBCF14F0030EDBCF15F0E750142649
:1028A000000E1522020E14C0DBFF030E15C0DBFF65
:1028B000020EDBCF14F0030EDBCF15F0D8901532EB
:1028C0001432020E14C0DBFF030E15C0DBFF898A31
:1028D000020EDBCF14F0030EDBCF15F014C0F3FFB4
:1028E00015C0F4FF060EE15C02E2E16AE552E16E1A
:1028F000E552E7CFD9FF1200D9CFE6FFE1CFD9FFEC
:10290000070EE126030EDB6A040EDB6A050EDB6AA6
:10291000060EDB6A8B90050EDB6A140EF36E050E55
:10292000DBCFF4FFF350F45C05E2060EDB2A050E64
:10293000DB2AF3D7060EDB6AC96A9EA6FED79E96EF
:10294000C950DF6EC96A9EA6FED79E96010EC9CFFA
:10295000DBFFC96A9EA6FED79E96020EC9CFDBFF9B
:10296000DF50E66ED950030FE96EDACFEAFFE55289
:10297000E750EE6EED6A030EDBCF14F0040E14C0C8
:1029800015F0146A030E14C0DBFF040E15C0DBFF44
:10299000010EDB50E76E030EDBCF14F0040EDBCF2D
:1029A00015F0E7501426000E1522030E14C0DBFFAD
:1029B000040E15C0DBFF030EDBCF14F0040EDBCFDB
:1029C00015F0060ED89014361536E804FBE1030E18
:1029D00014C0DBFF040E15C0DBFF020EDB40E84035
:1029E0003F0BE76E030EDBCF14F0040EDBCF15F0C8
:1029F000E7501426000E1522030E14C0DBFF040E50
:102A000015C0DBFF8B80030EDBCF14F0040EDBCF91
:102A100015F014C0F3FF15C0F4FF070EE15C02E2ED
:102A2000E16AE552E16EE552E7CFD9FF1200D9CF56
:102A3000E6FFE1CFD9FF020EE126DE6ADD6AFE0E77
:102A4000DB501F0BF36EF346F346830EC214F310F4
:102A5000C26EC282C2B2FED7C450176E166AC3508D
:102A60001624146E000E172014C0DEFFDD6EDECFBC
:102A700014F0DDCF15F014C0F3FF15C0F4FF020E03
:102A8000E15C02E2E16AE552E16EE552E7CFD9FF8F
:022A9000120032
:0E2A9200006AE86A0EAE56EF15F00B6C0C1ED3
:102AA0000D1E0E1E0C220D220E22001E09AE61EF1D
:102AB00015F0066C071E081E091E072208220922AF
:102AC000001E22EC16F009BE78EF15F000AE000CE7
:102AD000066C071E081E091EE86A07220822092242
:102AE000026C031E041E051E032204220522000C94
:102AF00000BE68EF15F00188FF0C08C012F0085006
:102B00000D02F4CF07F0F3CF06F009500E02F4CF18
:102B100009F0F3CF08F00D02F3500726F450082215
:102B2000E86A092212500E02F3500726F4500822D8
:062B3000E86A0922000C16
:0A2B36001E0EF66E000EF76E000E84
:102B4000F86E02010900F550E86F0900F550E96FD1
:102B500003E1E86701D03DD00900F550E36F0900BB
:102B6000F550E46F0900F550E56F09000900F550D4
:102B7000E96E0900F550EA6E090009000900F550F8
:102B8000E66F0900F550E76F09000900F6CFEAF299
:102B9000F7CFEBF2F8CFECF2E3C2F6FFE4C2F7FFB7
:102BA000E5C2F8FF0201E65302E1E75307E009003E
:102BB000F550EE6EE607F8E2E707F9D7EAC2F6FF4E
:102BC000EBC2F7FFECC2F8FF0201E807000EE95B79
:042BD000BFD7120059
:0C2BD40006500B02F3CF02F0F4CF03F028
:102BE0000C02F3500326000EF420046E06500D0272
:102BF000F3500426000EF420056E06500E02F3502A
:102C0000052607500B02F3500326F4500422000E51
:102C1000052207500C02F3500426F45005220750F9
:102C20000D02F350052608500B02F3500426F45011
:102C3000052208500C02F350052609500B02F350F0
:042C40000526120053
:0C2C4400056A046A036A026A200EE76E4B
:102C5000D89006360736083609360236033604366B
:102C600005360B50025C0C5003580D5004580E50A2
:102C7000055809E30B50025E0C50035A0D50045ADC
:0C2C80000E50055A062AE72EE4D7120079
:042C8C00FF0EE35004
:102C9000266E480E01D04C0EE76EE72EFED7E76A8F
:0C2CA000E72EFED7262EF7D7000012000A
:042CAC00410EF36E74
:102CB00000EE00F00E0E01D81200EA6002D0EE6ABB
:0C2CC000FCD7F350E9601200EE6AFCD76C
:042CCC001DEE00F009
:102CD0002DEE00F0F86A019C9BEC15F003EC00F07F
:082CE000CAEC0DF0FBD7120055
:082CE800FF0EE350266E1B0EE7
:102CF00000D001D0200EE76EE72EFED7262EFAD7A1
:042D000000D01200ED
:0C2D0400000000000000000000000000C3
:102D1000000001000000200004010806010101007C
:072D200000000000000000AC
:020000040030CA
:0100000015EA
:0100010013EB
:0100030020DC
:00000001FF
